:020000040000FA
:100000002E288207003400340034003400341B34BE
:1000100077344034003435346734E03400346A34A3
:10002000CF34C03400349A341D3420340034D534F5
:100030009F34803401341334B234203401344034DA
:100040006F34403401347B34CA3490340134AB34DF
:100050003F3400340134C934C33480348B01073059
:100060009F00AC2383168113FB3085008601831229
:10007000AD01AE01AF01B001B101D022D022051116
:10008000CE20EE20D110051A4828D1140C22D11010
:1000900083169B0194231A088312BB0083169423B2
:1000A0001A088312BC00831694231A088312BD0019
:1000B000831694231A088312BE00831694231A0809
:1000C0008312A000831694231A088312A1008316BA
:1000D00094231A088312A200831694231A08831209
:1000E000A300EA2218239922D0220508CB0003306E
:1000F0004B05CA00C8014030C700CC01CF01A9217F
:10010000CB198428A4207F28B501B401B3010130A4
:10011000B2004B1A9528E830B2000330B30095289E
:100120000310B20DB30DB40DB50DC70DC80D031CF2
:100130009028CC189D2896219F2859217121EA22C8
:1001400018239922D0227F28CC18B0280430CF025F
:10015000D7304F07031CAE282830CF00BC20B7286B
:100160000430CF07D7304F070318CF01BC20EA2255
:1001700018239922D02208004F080120A300CF0A9B
:100180004F080120A200CF0A4F080120A100CF0A8A
:100190004F080120A0000330CF020800A323033042
:1001A00086000616A3230612033086000616A62331
:1001B0000612033086000616A623061202308600B9
:1001C0000616A9230612283065230830652301305E
:1001D0006523063065230C306523080080306523D5
:1001E00050306923493069234330692345306923FE
:1001F0004C30692367306923653069236E30692389
:100200008830C3006523363069232E3069233030AF
:1002100069232D306923363069233030692320303B
:10022000692320306923C030652341306923413080
:100230006923303069235A3069235A3069232030CA
:1002400069232F306923203069234B3069236130C3
:1002500069236E3069236730692361306923203058
:10026000692355306923533069239823C0306523AF
:10027000203069232030692320306923203069230E
:1002800020306923203069232030692320306923FE
:1002900020306923203069232030692320306923EE
:1002A00020306923203069232030692320306923DE
:1002B00008003208A007031C6229A10F6229A20FBF
:1002C0006229A30A3308A107031C6929A20F69291F
:1002D000A30A3408A207031C6E29A30A3508A30742
:1002E0000800FC30230703188D2903302302031C68
:1002F00095296C30220703188D2993302202031CA4
:1003000095297830210703188D2987302102031C95
:10031000952900302002031C95290030A000873069
:10032000A1009330A2000330A3000800B209B30972
:10033000B409B509B20FA129B30FA129B40FA1299E
:10034000B50A5921A31FA829A001A101A201A30157
:100350000800C8014030C700D11CD321C81BB429F4
:100360000830C7070318C80A0508CB0003304B053F
:10037000C9004A060319AC290310CA0D4908CA0668
:100380004A080239CD004C060319CB294D08CC0090
:100390004908CA00AC29CC01CA1CD0290230CC00C3
:1003A0004908CA000800051ED8298519E129DD2958
:1003B0008519DF295118E329F62951140B2A511008
:1003C0000B2AD1010B2A1030D200051AEC29A023E8
:1003D000D20BE52980220B2AB5010F30B400423040
:1003E000B3004030B20059217121072A1030D200E9
:1003F0008519FF29A023D20BF82980220B2AB501E9
:100400000F30B4004230B3004030B2009621EA22EF
:1004100018239922D02208008030A0009630A10035
:100420009830A2000030A30083169B0194231A0881
:100430008312BB00831694231A088312BC00831610
:1004400094231A088312BD00831694231A0883127A
:10045000BE00EA221823C430C30065234330C30022
:1004600069234130C30069234C30C30069239922BA
:10047000D022A921B501B401B3011030B2004B194B
:10048000432A8030B2000000CC18512AB209B309C7
:10049000B409B509B20F512AB30F512AB40F512A2A
:1004A000B50A3208BB07031C5A2ABC0F5A2ABD0FD3
:1004B0005A2ABE0A3308BC07031C612ABD0F612AF1
:1004C000BE0A3408BD07031C662ABE0A3508BE07EB
:1004D000051E372A3B0883169B019A008723831247
:1004E0003C0883169A00872383123D0883169A00DE
:1004F000872383123E0883169A00872383120800FD
:10050000831604309B008312200883169A008723E9
:100510008312210883169A008723831222088316E8
:100520009A0087238312230883169A008723831255
:100530000800AD01AE01AF01B001B1012030B8003B
:100540003B08BF003C08C0003D08C1003E08C20097
:1005500003103F1CC22A2008AE07031CB42AAF0FA9
:10056000B42AB00FB42AB10A2108AF07031CBB2A72
:10057000B00FBB2AB10A2208B007031CC02AB10A77
:100580002308B107B10CB00CAF0CAE0CAD0CC20C13
:10059000C10CC00CBF0CB80BA82A0130B100080078
:1005A0002D3084000008BA000830B900BA0C031CD2
:1005B000DD2A861506150611E02A86110615061194
:1005C000B90BD62A840A32300402031CD22A8617B9
:1005D000861308002030B600A801A901AA01AB01CA
:1005E000AC010310A00DA10DA20DA30D0318201442
:1005F000A80DA90DAA0DAB0DAC0DB603031D012B63
:100600000800283084000D23840A0D23840A0D235A
:10061000840A0D23840A0D23F12A03300007B70052
:10062000B719800030300007B700B71B8000080002
:1006300080306523203069232B0E0F39303E69232B
:100640002B080F39303E69232C3069232A0E0F39CD
:10065000303E69232A080F39303E6923290E0F39AD
:10066000303E69232E3069238830652329080F39ED
:10067000303E6923280E0F39303E692328080F3990
:10068000303E6923203069236B3069234830692369
:100690007A306923203069230800860183160830E8
:1006A0008600831206138616FF30C500061606085C
:1006B000C400061200000000061600000612C50362
:1006C0000319642BC419562B0800C300D00106136C
:1006D0006C2BC300501406174D238601831600307F
:1006E000860083128612061350180617F03086050E
:1006F000430E0F398604061600000612F0308605F8
:1007000043080F39860406160000061208001C155F
:100710008B1355309D00AA309D009C149C188E2B85
:100720009C171C119B0A08001C141A089B0A08003D
:100730009D239D239D239D230800A023A023080023
:10074000FF30C500AE2B8030C500AE2B4030C50059
:10075000AE2B2030C500AE2B1030C500FF30C600D8
:0A076000C60BB02BC50BAE2B080032
:02400E00303F41
:10420000DE006500DC00170028000100D600000079
:10421000000000000000000000000000000000009E
:10422000000000000000000000000000000000008E
:10423000000000000000000000000000000000007E
:10424000000000000000000000000000000000006E
:10425000000000000000000000000000000000005E
:10426000000000000000000000000000000000004E
:10427000000000000000000000000000000000003E
:10428000000000000000000000000000000000002E
:10429000000000000000000000000000000000001E
:1042A000000000000000000000000000000000000E
:1042B00000000000000000000000000000000000FE
:1042C00000000000000000000000000000000000EE
:1042D00000000000000000000000000000000000DE
:1042E00000000000000000000000000000000000CE
:00000001FF
